:02000000952841
:08000800FF00030E8301A000BC
:100010000A08A1008A010408A2000E280313831213
:1000200086181828FA0A04307A0603192128192894
:10003000FA0106183428FB0A04307B0603192B2822
:1000400035282830F400F201F501F60A3C30760636
:10005000031D3528F6012830F400F201F70A0C30B0
:1000600077060319F7013528FB010B1D8B280B11AF
:10007000FF308100F40A32307406031D5828013025
:10008000F202031846280230F200FC0AF401F50AD5
:100090003C307506031D5828F501F60A3C307606FB
:1000A000031D5828F601F70A0C3077060319F701EB
:1000B000F208031D6428FF3086000F3085007708A2
:1000C000F9007608F8008B287908721878088316EA
:1000D0009B001C1472187A28F908031D722812302C
:1000E0009A007A280A301A0203187A28F0309A0403
:1000F0007C189A0E1A08831286000F398500721830
:100100000517721C85174A30740783169B001C1450
:100110001A08831295008B162208840021088A0091
:10012000200E8300FF0E7F0E09008030F00040306B
:10013000F1000230F200F401F501F601F701F801D7
:10014000F901FA01FB01FC01FF30A400FF30A5001A
:100150003030D1200730CF208312031307309F00A7
:100160006400810183166F30810064006830810073
:100170008312FF30810083168E15FF3092008312A8
:10018000950197121712043092000F3097000B114F
:100190008B168B17CF3085000000CC28CE28A50009
:1001A000D328A400D6282508660008002408650086
:0201B000080045
:02400E00703F01
:024200000000bc
:024202000100b9
:024204000200b6
:024206000300b3
:024208000400b0
:02420a000500ad
:02420c000600aa
:02420e000700a7
:024210000800a4
:024212000900a1
:02421400100098
:02421600110095
:02421800120092
:02421a0013008f
:02421c0014008c
:02421e00150089
:02422000160086
:02422200170083
:02422400180080
:0242260019007d
:02422800200074
:02422a00210071
:02422c0022006e
:02422e0023006b
:02423000240068
:02423200250065
:02423400260062
:0242360027005f
:0242380028005c
:02423a00290059
:02423c00300050
:02423e0031004d
:0242400032004a
:02424200330047
:02424400340044
:02424600350041
:0242480036003e
:02424a0037003b
:02424c00380038
:02424e00390035
:0242500040002c
:02425200410029
:02425400420026
:02425600430023
:02425800440020
:02425a0045001d
:02425c0046001a
:02425e00470017
:02426000480014
:02426200490011
:02426400500008
:02426600510005
:02426800520002
:02426a005300ff
:02426c005400fc
:02426e005500f9
:024270005600f6
:024272005700f3
:024274005800f0
:024276005900ed
:0242800000003c
:0242820000003a
:02428400000038
:02428600000036
:02428800000034
:02428a00000032
:02428c00000030
:02428e0000002e
:0242900000002c
:0242920000002a
:02429400000028
:02429600000026
:02429800000024
:02429a00000022
:02429c00000020
:02429e0000001e
:0242a00000001c
:0242a20000001a
:0242a400000018
:0242a600000016
:0242a800000014
:0242aa00000012
:0242ac00000010
:0242ae0000000e
:0242b00000000c
:0242b20000000a
:0242b400000008
:0242b600000006
:0242b800000004
:0242ba00000002
:0242bc00000000
:0242be000000fe
:0242c0000000fc
:0242c2000000fa
:0242c4000000f8
:0242c6000000f6
:0242c8000000f4
:0242ca000000f2
:0242cc000a00e6
:0242ce001500d9
:0242d0002100cb
:0242d2002e00bc
:0242d4003b00ad
:0242d60049009d
:0242d80057008d
:0242da0065007d
:0242dc0073006d
:0242de0081005d
:0242e0008e004e
:0242e2009c003e
:0242e400a80030
:0242e600b40022
:0242e800bf0015
:0242ea00c90009
:0242ec00d200fe
:0242ee00da00f4
:0242f000e000ec
:0242f200e500e5
:0242f400e900df
:0242f600eb00db
:00000001FF
